:020000040800F2
:10500000581A0020D550000859820008557A000827
:105010000000000000000000000000000000000090
:10502000000000000000000000000000D58B000818
:1050300000000000000000003D8A0008D18C00083C
:10504000E7500008E7500008E7500008E750000864
:10505000E7500008155B0008E7500008E75000081B
:1050600000000000E7500008515A0008E75000080F
:10507000E7500008B57E000800000000E750000877
:1050800000000000E75000080000000000000000E1
:10509000E750000800000000E7500008E750000853
:1050A000E7500008E7500008E7500008099400089E
:1050B000E7500008E7500008000000000000000072
:1050C0000348854600F060FC00480047D9A100086D
:1050D000581A00200448804704480047FEE7FEE7CE
:1050E000FEE7FEE7FEE7FEE76D8D0008C150000811
:1050F00030B50B46014600202022012409E00D4670
:10510000D5409D4205D31D469540491B25469540F7
:1051100040191546521E002DF1DC30BDF0B51FB40C
:105120000646002082B005464024019100901BE015
:10513000019922460F46304600F04EFB049A059B2B
:10514000801A994110D310461946224600F034FBCC
:10515000361A8F410197224601200021009F00F05E
:105160002BFB38184D4100902046641E0028DFDCE0
:10517000019B00982946324607B0F0BD03460B4319
:105180009B0703D009E008C9121F08C0042AFAD2FD
:1051900003E00B780370401C491C521EF9D2704783
:1051A000D2B201E00270401C491EFBD270470022BF
:1051B000F6E710B513460A4604461946FFF7F0FF16
:1051C000204610BD30B504460020034600E05B1CBD
:1051D000934203D2E05CCD5C401BF8D030BDF8B503
:1051E00002464A40D40F42004B0052085B089A42E4
:1051F00002D20246084611464A0023D0C30D4A0097
:10520000DDB2120EAD1A202D35DA49020126490A07
:10521000F6058A19002C00D0524220214F1B11465E
:10522000B9402A411018C20D9A4221D0002C17D043
:10523000012D08DCDA05801AD20F8019D207DBB203
:1052400000F0F6FAF8BDDA05801A012340001B06CB
:10525000C01880185A428018CA0F1043490007E04E
:105260004908C2071143DA05801A801940088018DE
:1052700000F0D6FAF8BD61000122511A001BF7E7D1
:105280000122D2075140AAE70122D2075040A6E7E7
:1052900070B502464A40D50F40004A00ED0740086D
:1052A0005208002814D0002A12D0C40DD30D410298
:1052B0000120C0055202490A520AE41A09181218BC
:1052C0007D34914201D3641C00E04900002C01DAD6
:1052D000002070BD0023914201D3891A0343400886
:1052E00049000028F7D100290AD0914202D10121BA
:1052F000C90705E0914201D2012101E00121C94322
:10530000E005C018401900F08BFA70BDF0B50746F3
:105310000846584087B0C00F049048000E46590018
:1053200040084908BC1A884105D2384631461E4615
:1053300017460B4602465800400810434CD0300D2B
:10534000039040055900400D490D0590401A029008
:10535000402872DA18030121000B09050843019067
:1053600004980092002805D00199524200208841FB
:1053700000920190029840210A1A0199009800F0C9
:105380001BFA05460C466B4607CB00F036FAC019EF
:105390007141039A0E0D0023D71756401A467A40E2
:1053A000164344D0049A002A2DD0029A012A039A67
:1053B00015DC1205C01A914101263605001C714109
:1053C000D20F059ED2070093019202962A462346E9
:1053D00000F074FA07B0F0BD38463146FAE716051A
:1053E000224A0F46B218C01AB74101210905001C14
:1053F0004F4100187F41114618187941E20F1043C0
:105400006D19644113E0E2076D0815436408C20793
:105410001443039A01261205C01A91413605001C57
:105420007141CE07400830434908C01851412A460F
:10543000234600F036FACDE7FFE70498012240004A
:10544000C117121A00238B4104983146C417381A29
:10545000A141EEE730B40124E407634030BC55E7D6
:1054600030B40124E407614030BC4FE70000E0FFA6
:10547000F0B51FB488B00B990998002448400999E9
:10548000C00F490049080991C0070B9900904900D5
:1054900049080B9109990898A64608431CD00B9916
:1054A0000A98084318D0099801244000420D48008A
:1054B000410D099824050003000B204309900B9827
:1054C0000003000B20430B9050181C494018002289
:1054D00001901446104605E0002001460DB0F0BDD5
:1054E000032801DA034600E003239C46C11A0AAEF2
:1054F0000AE05F0008ADED5B4F00F75B7D430027DE
:10550000AA187C41491C5B1E6145F2DD410004ABD9
:105510005A522104120C0A43240C401C0828DFDBD9
:10552000019802900099704601910090059B049AA1
:105530000799069800F0C2F9D0E700000DFCFFFFC4
:10554000F0B50C465C4085B0E40FE40703944C00D2
:1055500000266408590094464908024602962243F0
:1055600021D062460A431ED06200570D4A000E0346
:105570002303550D012402462C492405781B1B0BDF
:10558000360B401823432643614600901C46501AB0
:10559000B44103D30098401C009002E09218009898
:1055A0005B41002803DA0020014605B0F0BD002071
:1055B000012109050746864611E064461D46141B75
:1055C000B54106D36546521BB341744607430C43AD
:1055D000A646CD0740084908284392185B41054676
:1055E0000D43EAD11046184313D060461946504087
:1055F0007140084306D06046101AB34106D201221A
:10560000002306E000220123DB0702E00122D2434F
:105610005310009874460105381C6141029C039D9B
:105620000019694100F03DF9BFE70000FD030000EB
:10563000C217C10F504010B54018CA079623002169
:1056400000F0F6F810BD10B500229623114600F0C8
:10565000EFF810BD0EB5C217C10F5040CA07401871
:105660000021054B0293019200910A460B4600F07F
:1056700025F903B000BD0000330400000EB5054954
:105680000291002100910A460B46019100F016F9A3
:1056900003B000BD33040000410040020122400A73
:1056A000D205090E80187F2901DA0020704796295B
:1056B00003DC9622511AC8407047963988407047DB
:1056C00070B5CD0F4A0009030123090B1B051943CF
:1056D0000B4BED070024520D9A4201DA002070BDF9
:1056E000074B34339A4203DC9A1A00F075F802E053
:1056F0000449511888402C43F1D0404270BD00004D
:10570000FF030000CDFBFFFF4A0009030123090B43
:105710001B051943094B10B5520D9A4201DA0020BE
:1057200010BD064B34339A4203DC9A1A00F054F849
:1057300010BD03495118884010BD0000FF03000050
:10574000CDFBFFFFC20FD207400040080BD0C10DB8
:105750000723DB01C91840020905400A1143C208AA
:10576000400711437047002001467047CB0FDB070D
:10577000490010B5490802460A4307D00A0D07241C
:105780000903E401090B121B002A01DC002010BDF3
:10579000C900440F0C43C100E018D205801800F086
:1057A0003FF810BD0122D207002800DB101A0029A3
:1057B00000DB511A8142704710B5202A04DB0146F4
:1057C000203A9140002010BD914020239C1A0346AE
:1057D000E3401943904010BD10B5202A04DB084671
:1057E000203AD040002110BD0B46D340D0402024A9
:1057F000A21A91400843194610BD10B5202A06DBB5
:10580000CB170846203A1041C1170B4306E00B4660
:105810001341D0402024A21A91400843194610BDDC
:10582000002904DA401C490001D1400840007047BB
:1058300070B40024050C05D11024000402D1002905
:1058400021D01124050E01D100020834050F01D129
:105850000001241D850F01D18000A41C002801DB5C
:105860004000641C002908D020252E1B0D46F54061
:10587000A14000D001212943084301061B1B000A57
:10588000DB1D02D5002070BC7047DB05181880189E
:105890000029F8DA401C4900F5D170BC40084000EE
:1058A000704710B5002B08DA0024401C61419218A3
:1058B0005B411A4301D14008400010BDF0B51FB450
:1058C00082B005460C0003D0084603F05BFE02E000
:1058D00003F058FE20300246009021462846FFF78C
:1058E0006BFF049B059A04460F4618431143084377
:1058F00014D0184610431BD0009840210A1A1846AD
:105900000599FFF769FF05460E46009A0599049828
:10591000FFF752FF084305D0012004E02046394636
:1059200007B0F0BD0020C11705430E432C43374399
:1059300000990E986305401A7905E40A00220C4389
:10594000FD0A0A3002D500200146E9E701051019D9
:1059500069410C9C0D9D00196941FFF7A2FFDFE72B
:1059600010B5002904DB0124E40740428C412146A4
:10597000002B04DB1C460123DB075242A341994262
:1059800000D1904210BD0000064C0125064E05E0F6
:10599000E36807CC2B430C3C98471034B442F7D350
:1059A000FFF792FB5CA500087CA5000838B504460B
:1059B000064805490068FFF79BFB604300E0401E76
:1059C00000900028FBD138BD40420F00EC000020C1
:1059D000F8B50446006881688907890F012902D15A
:1059E0000168C90722D18168114A1026114001259A
:1059F00000290ED18168294381600120FFF7D6FF7D
:105A000000F098FF07460CE000F094FFC01B0A2846
:105A100007D9606D30436065A06D2843A065012003
:105A2000F8BD20680068C043C007EDD10020F8BD74
:105A30001700008010B500231A4603E0845CE318C9
:105A40009BB2521C8A42F9D3D84380B210BD0000E9
:105A500010B5034800F032FD024800F02FFD10BDE4
:105A6000F4150020AC15002030B5446C1C252C40EA
:105A70000125A540046C6560046863608368102B91
:105A8000036803D099600068C26030BD9A60006806
:105A9000C16030BD10490120487202205E31487259
:105AA00003203C39487204200E3948720A4B0B49D6
:105AB0005A1C0878587149789971233318715971B3
:105AC000203318775977107551751A461E321075A4
:105AD000517510765176704720110020D8000020B3
:105AE00010B503F04FF8202003F0E8F8012004F08F
:105AF000F9F8002003F0E2F8044803F097FF0448A7
:105B000004F040FA002004F075FA10BDA80000204F
:105B10008380000070B505200121000700F0FEFE23
:105B200000240D4D002800D02C6002210B4800F00D
:105B3000F5FE002808D10A482C6000880A21484355
:105B40000849088003F072FC012000F01FFE0220CB
:105B500000F01CFE70BD0000E400002000040050B6
:105B6000CC000020D60000207047000010B5084986
:105B700000224A6107494B684C1523434B604B6830
:105B8000082423434B60C009C001026010BD00001F
:105B90003C160020002002407FB500250C4606463A
:105BA000039500F0C3FDE009029003A9019600955A
:105BB000684600F053FD002804D000F08BFD002063
:105BC00004B070BD00F086FD0120F9E710B5002398
:105BD00002E0C45CCC545B1C9342FAD310BD0000BD
:105BE00010B5214A00219069C305204804D54169B8
:105BF000022319434161911593699B0505D54369BA
:105C00000124234343616302194393695B0505D56E
:105C10004369082423434361E301194393691B0546
:105C200005D54369042423434361630219439369FF
:105C30009B0405D543691024234343616302194340
:105C400093699B0304D5446920231C434461194391
:105C50009369DB0305D54369402423434361A002D4
:105C60000143916110BD0000002002403C1600205D
:105C700070B5054600F05EFE0646184C0AE0681C4A
:105C800008D0002D04D000F055FE801BA84201D999
:105C9000032070BDA069C007F1D1A069800701D5BC
:105CA0000220A061A069C00511D4A06980050ED4AE
:105CB000A06940050BD4A069000508D4A069800440
:105CC00005D4A069800302D4A069C00303D5FFF7FF
:105CD00087FF012070BD002070BD00000020024041
:105CE000F8B51746002605460C4600F01FFD09E0F2
:105CF00029460220226800F0FBFC002804D1241D64
:105D00002D1D361DBE42F3D300F0E4FCBE4201D28D
:105D10000020F8BD0120F8BD10B50849024600205A
:105D2000054B497905E044001C5B944203D0401CBC
:105D3000C0B28842F7D310BD621200204800002094
:105D400010B5094800F098FF80B2FFF797FC074AAA
:105D5000074BFFF78DFB0022064BFFF7F1FBFFF728
:105D6000D3FC80B210BD0000A4140020F853E3A5BA
:105D70009B843E4000408F40F8B5404CE0790028BD
:105D800001D0002000E00120E0713C493C48CA7984
:105D90000275097A41753B490A780276497841765D
:105DA0003749052013314872962004F0DBF84B2068
:105DB000C00004F0F1F83249002213310C2004F045
:105DC000BBF900210C2004F0C9F9022004F01AF9F3
:105DD0002D4D00210F2004F03FF82842E062F8D05A
:105DE000E06A411C3BD0294E294F400439D581221D
:105DF000D20100210F2004F074F90021102004F0DA
:105E00002BF841061E48490E0022633004F05AF870
:105E10001B4D6335687A052820D102221949681D77
:105E2000FFF7D0F9002819D1A87A6071134804222D
:105E3000691C4030FFF7A2F9206C00F02DF8608358
:105E40006079294642000B3108467330FFF796F916
:105E5000608B31884843388002202070F8BD02F002
:105E60001FFA0C480188608B0546FFF741F930881E
:105E7000414339806D1E6583F8BD00004800002055
:105E800081110020D800002000D02724C600002067
:105E9000C4000020C800002010B504460E4800F0E1
:105EA000EBFE0E49C006C00E098805E02246C2403E
:105EB000D2070FD0401CC0B28842F7D3012005E0C2
:105EC0002246C240D20705D0401CC0B28842F7D358
:105ED000491EC8B210BD0000A4140020C800002054
:105EE00010B5084800F096FA0A21064800F032FA88
:105EF000044800F01DF9800503D5024800F01AF9A6
:105F000080B210BD48140020F8B52F4D00220121A9
:105F1000284600F008FDFFF7E3FFFFF794FB2B4E48
:105F20003146FFF7B5F92A4C0122A06011462846F8
:105F300000F0F9FC2749A068002588423EDB207864
:105F4000254F002815D02570FFF7CAFFFFF77BFB10
:105F50003146FFF79DF9A060FFF7F4FB00223B46B6
:105F6000FFF778FA00221D4BFFF782FAFFF7FEFBDE
:105F70006060A068FFF7E6FB00223B46FFF76AFA85
:105F8000174A184BFFF774FA06460F466068FFF78A
:105F9000D9FB134A144B5242FFF76AFA32463B468A
:105FA000FFF7B4F9FFF7E2FB10496060884201DDBA
:105FB000616004E0FF21C905C84200D365606068E4
:105FC000FFF76AFBC0B2F8BD0004005000401B445C
:105FD000240000200000604000000C4000E064400D
:105FE0003333333333B33040CCCCEC3F0000C842C2
:105FF000F8B5054604464035287C0026012808D01F
:1060000001202874206881688907890F01290ED131
:1060100001E00220F8BD0168C90708D0606D2021A9
:10602000084360650126002028743046F8BD616D84
:10603000FF2201329143022211436165C168890741
:10604000890F0091C16889088900C1602068816852
:1060500092071143816000F06DFC07460EE000F0EE
:1060600069FCC01B0A2809D9606D022188431021F0
:1060700008436065002028740120F8BD206880680E
:106080000028ECDB2068C168009A1143C160606D94
:1060900080088000401C6065C5E70000F8B5064632
:1060A0000D464036317C01290DD001213174016843
:1060B0008A68520709D5416D2022114341650020AD
:1060C00030740120F8BD0220F8BD174B6A68D8056E
:1060D00047109A42154C8A6A2B6812D05B035B0BFF
:1060E0001A438A622968490305D5A1680143A16062
:1060F0000A20FFF75BFC2868800312D5A0683843AC
:106100000EE05B035B0B9A438A622968490302D560
:10611000A1688143A1602868800302D5A068B843C4
:10612000A06000203074F8BD01100000002701407D
:10613000406D70470068006C7047000070B5040047
:1061400006D0606D264600254036002802D006E0C5
:10615000012070BDA5653574204600F0D3F8606D50
:10616000C00603D421688868400705D5606D1021FA
:10617000084360653574EBE7606DFF2201329043A0
:1061800002221043606588688207920F5B48012AEB
:1061900002D10A68D2072BD1032362689B079A4277
:1061A00005D05B429A4202D05B009A4209D10A694B
:1061B000920092080A6121680A6963681A430A61B9
:1061C0000CE00A69920092080A6181680F22920429
:1061D0009143816081686268114381602168CA6867
:1061E00018239A43CA602168CA68A3681A43CA6020
:1061F000816801225206914381608168A28E520615
:106200001143816020688168C90004D4816801223B
:106210001207114381602068C168394A1140C1608A
:106220002069E168022825D0002001432046203063
:106230000278037B52035B001A431143226B114324
:10624000A26992031143E269D20311432268D36821
:106250001943D160616A0A46FF3AC23A05D0A26A80
:1062600011432268D3681943D16042780121012A81
:1062700002D00BE00420D8E70078002823D0606D1E
:10628000202210436065A06D0843A065E06B0128E3
:1062900020681FD00169C90703D001694908490076
:1062A000016120684169C908C900416120684169EC
:1062B000A26B11434161A565606D80088000401CA0
:1062C0006065002070BD2068C26801231B041A436A
:1062D000C260DBE70269FF239B009A4302612068EA
:1062E0000269236CA66C1A43636C33431A43026140
:1062F000206802690A430261D3E7000000270140D9
:106300001902FEFF10B586B0044614216846FEF758
:106310004EFF0E492068884216D10D48416B421548
:1063200011434163C16A01221143C162C06A6946D7
:106330001040059002200090032001900020029060
:106340000520000700F02EFA06B010BD0024014021
:1063500000100240F8B504464069254640350E4617
:1063600008280BD02068C068C00709D0606D2021C4
:1063700008436065002028740120F8BD082700E06C
:106380000C2700F0D7FA009011E0701C0FD0002EFF
:1063900005D000F0CFFA0099401AB04207D9606DDD
:1063A000042108436065002028740320F8BD20689C
:1063B00000683842E9D0606D0121490208436065F8
:1063C0002068C16809058A0F0C21002A1BD12022F0
:1063D000125D002A17D10268120714D5826853078C
:1063E0000122002B08DB43688B434360606D13027E
:1063F00098431043606506E0606D20231843606594
:10640000A06D1043A065A069002801D1206801603B
:106410000020F8BD70B5044621680020896849074E
:1064200021D425464035297C01291CD0012129741D
:10643000E169012904D02046FFF7CAFA002811D1EA
:10644000616D0A4A1140FF2201321143616500214A
:10645000A165297422681C21116021688A680423BF
:106460001A438A6070BD022070BD0000FEF1FFFF7C
:1064700070B50024014620314A79022A03D0042154
:10648000C163012418E0026813680E25AB43136052
:10649000026813685B085B001360436C1C221340A6
:1064A000012215469D40036C5D604A7100220A710D
:1064B000816B002900D08847204670BDF0B4016C84
:1064C0000D6801680C68466C1C2304221E401746A8
:1064D000B7402F420ED067070CD50C68A40602D433
:1064E0000C6894430C60416C19408A40016C4A600E
:1064F000016B1AE00227B74002462F402032002FDE
:1065000017D0A70715D50C68A40605D40C680A2572
:10651000AC430C6001215171446C02211C40036C9E
:10652000A140596000211171C16A002918D0F0BC46
:1065300008470827B7402F4212D0240710D50C680F
:106540000E25AC430C60446C01211C400B46A3405B
:10655000046C6360C163517100211171416BE4E708
:10656000F0BC704770B504003CD01F48256814216A
:106570002818FEF7BDFD800060641C4820640221DD
:10658000204620300246417129681948E3680140DD
:10659000A06866691843236933431843A369184305
:1065A000E3691843236A1843084328600121A0685F
:1065B0008903884210D00D488030836A656C1C21A5
:1065C0000D400F26AE40B3438362656C63680D4097
:1065D000816AAB400B4383620020E063012151716B
:1065E000107170BD012070BDF8FFFDBF00000240BA
:1065F0000F80FFFFF8B504468C4620300179002556
:10660000012909D00126067141790027012905D009
:10661000077102252846F8BD0220F8BD022141710C
:10662000E763206801684908490001606146204627
:10663000FFF71AFA206B00282068016801D00E22AB
:1066400005E0042291430160206801680A22114399
:1066500001602068016831430160DBE7F8B51A4E3C
:106660000546307C0F46012807D0012030741748BA
:10667000FFF7FEFA010002D021E00220F8BD002061
:10668000C04338606C6814E02046FFF76FFA0F488B
:10669000FFF7EEFA01460E48426808239A4342602B
:1066A000426843159A434260002901D03C6006E0ED
:1066B0008034A8686A68C0018018A042E4D800202D
:1066C00030740846F8BD00003C16002050C300009E
:1066D00000200240054841680222114341604168A0
:1066E0000122114341600020704700000020024059
:1066F000F8B50C4C1646207C0F46012808D0012026
:1067000020740948FFF7B4FA0025002802D006E0FB
:106710000220F8BD65613E600348FFF7A9FA2574C1
:10672000F8BD00003C16002050C30000114841682D
:10673000C9070BD0EFF3108172B60F4AC2600F4A3F
:10674000C26081F310884168C9070ED1416889078A
:106750000DD5EFF3108172B6094A0261094A026150
:1067600081F310884068800701D501207047002020
:106770007047000000200240EFCDAB890504030202
:10678000BFAE9D8C161514137047000010B5044958
:106790004A69024202D04861FFF7F6FF10BD0000CF
:1067A00000040140F8B500230124A2E027469F40E1
:1067B0003A4070D04D68022D01D0122D14D1DD0861
:1067C000AD002D1800952D6A5E07AC46F50E0F261C
:1067D000AE46AE406546B543AC460E697546AE4022
:1067E00065462E43009D2E624D68012D05D0022D79
:1067F00003D0112D01D0122D16D185680326AC4689
:106800005D00AE46AE406546B543AC46CE687546C3
:10681000AE4065462E43866046680D79BE43ED0660
:10682000ED0F9D403543456006685F000325BD4080
:10683000AE46AE430D79B446AE07B60FBE406546D0
:106840002E430660C6687546AE438D68BD4035432D
:10685000C5604D68ED004BD5294D6E6B26436E63C8
:106860009E08284DB6007519AC46AD689E07360FD8
:106870000F27B740BD4305273F07B84201D1002786
:1068800015E0214FB84201D1012710E01F4FB84257
:1068900002D102270BE02BE01D4FB84201D10327A4
:1068A00005E01C4FB84201D1052700E00627B7409C
:1068B0002F436546AF60184D2E684F689643FF031F
:1068C00000D516432E606E684F689643BF0300D50F
:1068D00016436E60AE684F689643FF0200D51643BC
:1068E000AE60EE684F689643BF0200D51643EE6077
:1068F0005B1C0A681546DD4000D057E7F8BD000074
:106900000010024000000140000400500008005048
:10691000000C0050001C00500004014000690840B9
:1069200000D001207047002A01D081617047816248
:10693000704700000148006870470000E800002030
:1069400002480168491C016070470000E80000200F
:1069500010B5084800240168402211430160204618
:1069600000F00AF8002801D0012401E000F0B0F99D
:10697000204610BD0020024070B5054609487D2123
:106980000024C9000068FEF7B3FB00F045FE0028B4
:1069900001D0012404E000222946501E00F0B8F97D
:1069A000204670BDEC00002070477047F8B52C4CB5
:1069B00001266078401C6070E670208B401C2083AC
:1069C000208902F045F9274DE888FEF73CFE26496C
:1069D000FEF75EFC254F3968FEF701FC38600221A6
:1069E0002348FFF79BFF002809D0002020621F48A2
:1069F0002049076820488F4212DD067012E0E888BF
:106A0000FEF721FE1849FEF743FC216AFEF7E7FB7B
:106A10001A4920628842EADB1A491948C860E6E749
:106A200000210170688F401EFEF702FE3946FEF716
:106A3000B9FE06D82079002803D01348C179314324
:106A4000C171688FFEF7FFFD08490968FEF7AAFECD
:106A500004D22079002801D003F054FCF8BD0000D6
:106A6000BC000020200D002000007A44E40000203B
:106A700000040050000040404E0000200000A040F4
:106A80000400FA0500ED00E094110020704770B595
:106A900005000DD002202C462034A073284601F0BA
:106AA00011FA284600F0BEF80020A073607370BD94
:106AB000012070BD7047704710B50446006801683A
:106AC000C943C90708D18168C943C90704D1012155
:106AD00041602046FFF76AFF20680168C9438907C3
:106AE00008D48168C943890704D402214160204643
:106AF000FFF75AFF20680168C943490708D4816835
:106B0000C943490704D404214160204600F0DEF85F
:106B100020680168C943090708D48168C943090787
:106B200004D4082141602046FFF7B0FF20680168C7
:106B3000C943C90608D48168C943C90604D41021D1
:106B400041602046FFF731FF20680168C94389068C
:106B500008D48168C943890604D4202141602046B5
:106B6000FFF7A9FF20680168C943490608D4816876
:106B7000C943490604D4402141602046FFF79AFFEB
:106B800010BD0000F8B5040005D025462035A87BCF
:106B9000002802D006E00120F8BD002068732046DE
:106BA00000F052F80220A8732068C2688446636827
:106BB000012B04D00120A16AC005814201D11E2011
:106BC000824315486169814201D01448024014484B
:106BD000A668024018463043676A266A3E4330433F
:106BE000A66A30431043012B03D00122D2059642FE
:106BF00003D12369E2681A431043074A914205D042
:106C0000A2691143E2690243084610436146C86025
:106C10000120A8730020F8BDFFFF00003F1FFFFF09
:106C2000F8F119FF10B500680549884207D10548F9
:106C3000816B4900490881630D2000F055F810BDB3
:106C4000007C00400010024010B5006808498842EE
:106C50000CD10848816BC2041143816300220121D9
:106C60000D2000F055F80D2000F048F810BD000090
:106C7000007C0040001002400068C06970470000BE
:106C800070B50224034620339C730F4C2568E6043C
:106C9000354325600468E568B6123543E56005684C
:106CA000AE6801242643AE6005682E6926432E6136
:106CB0000568A96101684A610068016904221143FD
:106CC00001619C73002070BD00040140704700000A
:106CD0000448416B012211434163816B020411435B
:106CE0008163704700100240C106C90E0120884030
:106CF000014908607047000080E100E0C106C90E4C
:106D000001208840014908607047000000E100E070
:106D100010B501F0A3FA10BD02494A6882434A60E7
:106D2000704700000070004002480168821511435E
:106D3000016070470070004002494A6802434A609F
:106D400070470000007000400548016802221143AE
:106D500001600448016904221143016130BF70479A
:106D60000070004000ED00E00A4B1A6892089200A3
:106D700002431A600848036904221343036101298E
:106D800006D040BF20BF20BF016991430161704719
:106D900030BFF9E70070004000ED00E0F8B50446B0
:106DA0000078544D800672D5524E0027403EB06B9D
:106DB000C00004D4B06BA9050843B06301274E4856
:106DC0000168C90511D40168821511430160FFF7FC
:106DD000B1FD009005E0FFF7ADFD0099401A642871
:106DE00037D845480068C005F5D532680321090544
:106DF00060680A400140914208D08103890F03294D
:106E000004D13168890301D50120F8BD2A69032125
:106E100009040A4022D0084090421FD02078800602
:106E20001CD528692A6988430121C9040A432A61BB
:106E30002A698A432A612861C0050FD5FFF77AFDC8
:106E4000009008E0FFF776FD0099411A2B48814237
:106E500001D90320F8BD28698005F3D5616888034E
:106E6000800F032805D132680005824301400A43A0
:106E700032602869032261681204114008432861C6
:106E8000002F04D0B16B012000078143B16320784B
:106E9000C00705D0E868A168800880000843E86062
:106EA0002078800705D5E8680C218843E16808430D
:106EB000E8602078400706D5E86803218902884306
:106EC00021690843E8602078000706D5E8680321B7
:106ED0000903884361690843E8602078000606D505
:106EE000E868032189048843A1690843E860002019
:106EF000F8BD000040100240007000408813000000
:106F0000F8B50E4605007DD053480068C007C00F95
:106F1000B0420AD250480168490849003143016033
:106F20000068C007C00FB04271D128784B4C800771
:106F300005D5E068F0218843A9680843E060287817
:106F4000C00752D06868022817D0032818D02168DB
:106F5000012818D08905002959DAE16889088900D3
:106F60000143E160FFF7E6FC69680746022912D099
:106F700003291CD0012926D033E021688903EAE7E0
:106F800021688901E7E74907E5E7FFF7D3FCC11B63
:106F90003348814223D8E0680007800F0228F4D1EB
:106FA00023E0FFF7C7FCC11B2D48814217D8E068DA
:106FB0000007800F0328F4D117E0FFF7BBFCC11BCB
:106FC000274881420BD8E0680007800F0128F4D1E0
:106FD0000BE0FFF7AFFCC11B2148814201D9032020
:106FE000F8BDE0680007800FF3D11B480168C907AE
:106FF000C90FB1420DD90168490849003143016008
:10700000006800E003E0C007C00FB04201D00120DB
:10701000F8BD2878400706D5E068072109028843B3
:10702000E9680843E0602878000707D5E068072191
:10703000C90288432969C9000843E06000F036F8B6
:10704000E168084A0906090F515CC8400649086012
:107050000020FFF791FCF8BD002002400010024024
:10706000881300003AA50008EC00002004480549F8
:107070000068C968044A4905490F515CC840704717
:10708000EC0000200010024053A500080448054908
:107090000068C968044A8904490F515CC8407047B8
:1070A000EC0000200010024053A5000810B5184A5B
:1070B000D1680C20084004280BD0082810D00C28D8
:1070C00010D050680004410F0120C003491C8840C3
:1070D00010BD1068C00601D50E4810BD0E4810BD89
:1070E0000E4810BD88020E4B000F185C0902D368D1
:1070F000890F491CDB0301D5084A05E01268D20656
:1071000001D5044A00E0044A5043FDF7F1FF10BDE9
:107110000010024000093D000024F40000127A0033
:107120004AA50008FEB505007ED0FE4CE7680C209D
:10713000E66807400120000406402878C00747D0D1
:10714000082F05D00C2F0AD101200004864206D159
:10715000206880033CD568680028E5D038E001202D
:1071600069680004814203D121680143216011E074
:10717000052301221B0492049942216802D1114384
:107180002160F1E78143216021680140009120687E
:1071900090432060686800280DD0FFF7CBFB00907B
:1071A00005E0FFF7C7FB0099401A64287AD82068E9
:1071B0008003F6D50CE0FFF7BDFB009005E0FFF77C
:1071C000B9FB0099401A6428F0D820688003F6D4EF
:1071D0002878800755D50923E868042F0DD00C2F97
:1071E00001D1002E09D000283BD0216899430143EA
:1071F0002160FFF79FFB064627E02168490701D57C
:10720000002891D061681F22120291432A6912025C
:10721000114361602168994301432160FFF746FFF4
:10722000E16809060A0F00E079E1BF49895CC840BE
:10723000BE4908600020FFF79FFB002872D120E0C4
:10724000FFF778FB801B0228B0D820684007F7D5ED
:1072500060681F21090288432969090208436060A8
:107260000FE02068400840002060FFF763FB0646FF
:1072700004E0FFF75FFB801B022897D820684007D7
:10728000F7D42878C0065FD5002F0CD0A869002855
:1072900049D02068FF21013108432060FFF74AFBF5
:1072A00006462DE0C0E02068800502D5A8690028C8
:1072B000A7D06068072149038843296A08436060B2
:1072C0006068297F0002000A090608436060286A96
:1072D000410B0120C003491C8840E16809060A0FE0
:1072E0009149895CC840914908600020FFF744FB40
:1072F000002817D128E0FFF71DFB801B0228A3D828
:1073000020688005F7D56068072149038843296A0A
:10731000084360606068297F0002000A090608438C
:10732000606011E0E1E02168FF20013081432160CD
:10733000FFF700FB064604E0FFF7FCFA801B02287B
:1073400072D820688005F7D42878794E000724D5B4
:1073500068690028306910D0012108433061FFF7C7
:10736000E9FA009005E0FFF7E5FA0099401A0228D3
:107370005AD830698007F6D50FE0400840003061E8
:10738000FFF7D8FA009005E0FFF7D4FA0099401A09
:10739000022849D830698007F6D42878400765D597
:1073A00000200290A06BC00006D4A06B0121090749
:1073B0000843A063012002905E480168C90511D40A
:1073C0000168821511430160FFF7B4FA009005E0EF
:1073D000FFF7B0FA0099401A642825D8554800688C
:1073E000C005F5D5FF20AA680130824203D131697A
:1073F0000143316111E001218902002A07D00523F0
:107400001B029A4203D132690A433261EFE73269C3
:1074100082433261306988433061A86800280FD008
:10742000FFF788FA009007E05EE0FFF783FA009923
:10743000411A4148814257D830698005F5D50DE0A1
:10744000FFF778FA009006E0FFF774FA0099411A06
:107450003948814248D830698005F5D4029800281F
:1074600004D0A06B012109078843A063686A002843
:1074700064D00C2F3ED0012636060228206805D0A5
:10748000B0432060FFF756FA05462FE0B043206076
:10749000FFF750FA074604E0FFF74CFAC01B02283A
:1074A00022D820688001F7D4E96AA86AE268084314
:1074B000296BFD231B049A4311430843E0602068B5
:1074C00030432060FFF736FA054604E0FFF732FA52
:1074D000401B022808D820688001F7D52EE0FFF76E
:1074E00029FA401B022801D90320FEBD2068800133
:1074F000F5D423E00128F8D0E06801210904AA6A44
:10750000014091420BD10F218904EA6A0140914266
:1075100005D1032189050840296B88420ED001203E
:10752000FEBD0000001002403AA50008EC0000205B
:107530004010024000700040881300000020EFE778
:1075400070B5040007D0002625464035A662687C49
:10755000002802D005E0012070BD2E74204600F006
:107560002FF802206874206801684022914301606E
:10757000A168606822690843E168114308436169B2
:1075800001220843A169520211400843E1690843FE
:10759000216A0843A16A084321680860A0690421A0
:1075A000000C0840616A0843216848602068C1698E
:1075B00092009143C161666501206874002070BD2E
:1075C00010B586B0044614216846FDF7F0FD104959
:1075D0002068884219D10F48416B821411434163DE
:1075E000C16A01221143C162C06A002110400590A6
:1075F000E02000900220019003200390029104916A
:10760000052069460007FFF7CDF806B010BD000061
:107610000030014000100240094910B5401E884268
:1076200001D9012010BD074C60610321081F00F043
:1076300015FE0020A06107202061002010BD000081
:10764000FFFFFF0000E000E070477047F8B50268F8
:107650000446D0691168936805072D0F5BD0DD07DC
:10766000ED0FFF2621360E402E4367D0C60706D009
:10767000CE0504D501261662E26F3243E267870722
:1076800002220426002F06DADF0704D027683A62B8
:10769000E76F3743E767470706D5DB0704D0236862
:1076A0001E62E36F1343E367020709D520220A40F5
:1076B0002A4305D0236808221A62E36F1343E36765
:1076C000E26F002A2FD0800606D5880604D5216EE9
:1076D000002901D020468847E06F21688968490663
:1076E00001D4000724D5204601F0FEFC2068816803
:1076F000490619D58168402291438160E06E0028D7
:1077000012D020498163E06EFEF7B2FE00280AD055
:10771000E06E816B06E0850610D58D060ED5216ED4
:107720001CE020468847F8BD2046FFF78EFFF8BDD5
:107730002046FFF78AFF0020E067F8BDC50208D5A4
:107740005B0206D50120000510622046FFF77CFF92
:10775000F8BD030605D50B0603D5616E0029E0D1FF
:10776000F8BD4006FCD54806FAD5136820464021EE
:107770008B431360202161670021616600F069F985
:10778000F8BD00004590000810B5040003D0606FFC
:10779000002802D007E0012010BD00217020015513
:1077A000204600F027F82420606720680168490817
:1077B00049000160204601F0E1FC0128ECD0606A3C
:1077C000002802D0204601F01FFB206841680922F2
:1077D000D20291434160206881682A2291438160EE
:1077E00020680168012211430160204601F072FB0C
:1077F00010BD0000F0B587B0064614216846FDF7BD
:10780000D6FC2C493068884251D12B48416B01226B
:10781000920311434163C16A01221143C162C06AEC
:10782000002510400590032040020090022003270D
:1078300001A9A1C104200490052069460007FEF7B4
:10784000B1FF1F4C1D48A560E56081C48027E5603D
:10785000A7602020256160610002A0611848083CF3
:10786000FEF780FE002801D0FEF77EF9F466A662DE
:10787000144C124821461438206003206060102008
:107880000831A1C16561A561E56120462562FEF769
:1078900069FE002801D0FEF767F9B46600220121D5
:1078A0001B20A662FFF734FA1B20FFF727FA07B068
:1078B000F0BD0000003801400010024030000240DE
:1078C000AC150020F4150020F8B50446806F202880
:1078D0004DD100290BD0002A09D00123A0681B0339
:1078E000984206D12069002803D1C80701D00120A1
:1078F000F8BD25466035287C012838D00120287441
:107900005820616502530026E6672220A067E06EDA
:10791000002819D01749C162E16E17480863E16E6B
:1079200016484863E06E13468663676D21683A46E1
:107930002431E06EFEF75EFE002805D01020E067DF
:107940002E7420206067D2E72E7420680168FF2221
:107950000132114301602068816801221143816076
:10796000206881684022114381600020F8BD022018
:10797000F8BD0000A1900008DF90000859900008B1
:1079800070477047FFB50446406F83B017460D46F9
:1079900020285CD1002D0AD0002F08D0A168C0019A
:1079A000814207D12069002804D1E80702D00120D4
:1079B00007B0F0BD204660300290007C012846D020
:1079C0000298012101740020E06721206067FEF722
:1079D000B1FF264640360190378277820120A168A8
:1079E0000003814202D12069002802D02F460025E1
:1079F00011E000270FE000228021204601F0D2FC98
:107A0000002815D1002F15D02168387888627F1C96
:107A1000708A401E7082708A019B00280698009030
:107A2000E9D100224021204601F0BCFC002808D00A
:107A30000320BDE728882168C005C00D8862AD1C01
:107A4000E6E720206067029900200874B0E7022072
:107A5000AEE7704701490248C160FDE70400FA053E
:107A600000ED00E010B50524240700220421204683
:107A7000FEF759FF002208212046FEF754FF0A2096
:107A800001F08DFF012204212046FEF74CFF0A2061
:107A900001F085FF002204212046FEF744FF10BDBF
:107AA00010B505242407002204212046FEF73BFFE1
:107AB000012208212046FEF736FF0A2001F06FFF61
:107AC000012204212046FEF72EFF0A2001F067FF65
:107AD000002204212046FEF726FF10BDF8B5002441
:107AE0000526074625463607002204213046FEF7C4
:107AF0001AFF0A2001F053FF012204213046FEF74D
:107B000012FF6006040E08213046FEF707FF00282A
:107B100001D0641CE4B2052001F041FF6D1CEDB200
:107B2000082DE1D3002F03D0FFF79CFF2046F8BDBE
:107B3000FFF7B6FFFAE770B50526054636070022BF
:107B400004213046FEF7EFFE0024E80901D00122AF
:107B500000E0002208213046FEF7E5FE6806050E2B
:107B60000A2001F01CFF012204213046FEF7DBFE53
:107B70000A2001F014FF002204213046FEF7D3FE54
:107B80000A2001F00CFF641CE4B2082CDDD370BDA8
:107B900010B505242407012208212046FEF7C3FE64
:107BA000012204212046FEF7BEFE002208212046C5
:107BB000FEF7B9FE0A2001F0F2FE00220421204661
:107BC000FEF7B1FE10BD10B50524240700220421E4
:107BD0002046FEF7A8FE002208212046FEF7A3FE5D
:107BE0000A2001F0DCFE012204212046FEF79BFE64
:107BF000012208212046FEF796FE0A2001F0CFFE62
:107C000010BD70B505252D07002401220821284646
:107C1000FEF789FE062001F0C2FE0122042128465B
:107C2000FEF781FE062001F0BAFE07E0641CE4B214
:107C3000FA2C03D9FFF7C7FF012070BD08212846A1
:107C4000FEF76CFE0028F1D1002204212846FEF741
:107C50006AFE002070BD0000F8B501F06BF901F07C
:107C6000A5F949480068C069484E494F800700D5CA
:107C7000FE60FEF765F8474C012162798902464DA6
:107C8000002A20D0454A1278002A1CD0012A04D0AC
:107C9000022A06D0032A08D115E0FF22F5329042CD
:107CA00011D200222846FEF73EFE0121C9023A48C1
:107CB000FEF734FE0025002826D039480560A0795B
:107CC000002802D005E00122ECE70120A07101F0BC
:107CD000ADFB2078632806D9002208212E48FEF744
:107CE00022FE012205E0012208212B48FEF71BFE9F
:107CF000002201210520C9030007FEF714FE294CCC
:107D0000A08C012803D01CE0A5710022ECE72648D6
:107D10006946088072B680212448FDF73DFF00289F
:107D200004D0022269462148FDF7DAFF62B620A09E
:107D300001F018FCA58402F081FB642001F028FE0C
:107D4000FE60608C012809D11648658440380580A2
:107D500002F074FB642001F01BFEFE60208C012801
:107D600006D1258402F06AFB642001F011FEFE605A
:107D70000C48134A40380188914202D1C08800283B
:107D800000D1FE60F8BD00002C1500200400FA05AB
:107D900000ED00E0BC000020000400505A0000206C
:107DA000E4000020600D0020AAAA0000384A000864
:107DB000BDF8C8EBC9FDBCB6C4A3CABD0D0A00001E
:107DC000AA55000008B53721202000F06EF80321E5
:107DD000212000F06AF84021222000F066F80821F6
:107DE000232000F062F8AA21302000F05EF80A4853
:107DF00002210187322000F058F80121332000F0E1
:107E000054F85F21202000F050F8684600F006F892
:107E10000A2001F0C4FD08BD200D002010B5014668
:107E20000F2000F021F8002800D0012010BD10B56F
:107E30000446FFF7ADFE3220FFF77DFEFFF7E1FEBF
:107E4000E0B2FFF778FEFFF7DCFEFFF7A1FE33207C
:107E5000FFF771FEFFF7D5FE0020FFF73FFE044657
:107E6000FFF7B1FE204610BD10B50C46FFF7DFFF4F
:107E70002070012010BD70B50D460446FFF788FE46
:107E80003220FFF758FEFFF7BCFEE0B2FFF753FECB
:107E9000FFF7B7FE2846FFF74EFEFFF7B2FEFFF7EB
:107EA00092FE0A2001F07BFD70BD10B5FFF7E3FFE5
:107EB000012010BD10B50248FEF7FEFD10BD000008
:107EC000A4140020FEB50446002572B60068394AA5
:107ED000831804D13849CD68032189040D40816895
:107EE0000191C168009141698669002B08D132482F
:107EF0004038836AC7043B438362836ABB4383621F
:107F00000846304348D02B482368C34205D12A484D
:107F1000C368032292049343C360002917D02068EA
:107F2000026901231A43026120684161FEF702FDE4
:107F30000746FEF7FFFC2168C01B0968090703D448
:107F40007D21C9008842F4D9216808204860002EAC
:107F500017D0206801690122114301612068866100
:107F6000FEF7E8FC7D270646FF00FEF7E3FC2168EC
:107F7000801B0968C90601D4B842F6D921681020CF
:107F800048600C482168C14206D10B48C1680322F1
:107F9000920491432943C16020680169490849005E
:107FA000016121680198886021680098C86062B604
:107FB000FEBD00000084FFBF401002401CB5002140
:107FC00016480091144A01910260C1631205426093
:107FD000816007228263012202610246C160203271
:107FE0001170FF235170C2334362816211730163C8
:107FF0008161042241634261C161FEF79FF8084834
:1080000000908013019069460448FEF747F800216C
:108010000248FDF7EDFF1CBD00240140481400207C
:108020000200000408B50848016B012211430163F6
:10803000006B01211040009000220A20FEF768FE2C
:108040000A20FEF75BFE08BD00100240F0B587B0C5
:1080500014216846FDF7ABF84C48C26A04210A4374
:10806000C262C26A0A400592C16A80273943C1626E
:10807000C16A39400591C16A01252943C162C16ABB
:1080800029400591C16A02263143C162C06A2A466D
:108090003040059005201C210007FEF744FC01221A
:1080A0003B493C48FEF73FFC00223B493948FEF77C
:1080B0003AFC91210520002209020007FEF733FC5B
:1080C0003648019000240520694600950294000777
:1080D000FEF768FB03200190052069460096029494
:1080E0000007FEF75FFB0C20009011200190032099
:1080F00003900520029469460007FEF753FB102009
:108100000090052069460396019502940007FEF74A
:1081100049FB1120019002946946009503941D4883
:10812000FEF740FB1E4801906946009602951948EB
:10813000FEF738FB1B4800900294694601950394B2
:108140001448FEF72FFBE8026A4651C269461148FF
:10815000FEF728FB9120000200900520029469465A
:10816000019503940007FEF71DFB69460948009737
:1081700002950194FEF716FB002201210520FEF76F
:10818000C7FD0520FEF7BAFD07B0F0BD00100240A4
:10819000010600000004005008300000000011102B
:1081A000000021100836000010B50F4C0D4820606B
:1081B000FF20053060600020A060E0602061606109
:1081C000E0610121206249026062A161A062072092
:1081D000E0622046FFF7B4F92068016840221143AD
:1081E000016010BD00300140D414002000B585B0FE
:1081F00014216846FCF7DBFF164815490160E121B0
:108200004902416000218160C160016181610C22ED
:10821000C161426101623021416201210903816330
:108220004900C163FFF7B0FA0120800200900220EC
:108230000190012002900320039004200490052067
:1082400069460007FEF7AEFA01F0EAF805B000BD96
:10825000003801402C150020704700008307FF22E2
:10826000DB0E9A408907090E994000280BDA0007B7
:10827000000F0838830808489B001818C369934307
:108280000B43C3617047830804489B001B181868A0
:10829000904308431860704700ED00E000E400E000
:1082A000BFF34F8F04490348C860BFF34F8F00BF2F
:1082B000FDE700000400FA0500ED00E0F0B58FB026
:1082C000962001F04FFE4B20C00001F065FEFF4CF0
:1082D00000256570A07B0C2801D30B20A073012220
:1082E000052051020007FEF71EFBA07B6073607142
:1082F000F748A570F74E007830710221F648FEF776
:108300000DFB002862D00020A179F24E49000843FD
:10831000F071A06AF070401CA06260793146B072C2
:108320004200CE310846C338FCF728FF06207072A1
:10833000304613380290217F0175617F4175607965
:108340000022400031460D3001F0F6FE6079002138
:1083500040000D3001F002FF022001F053FEF571E4
:108360002574A57201202073E572DC48FEF784FCB9
:1083700020840646A5706079FDF780F9D84AD94B6C
:10838000FDF776F801F0A0FA0022D74BFCF7BEFF0C
:10839000FDF7BAF90006C00C801980B20121C903AB
:1083A0006084884201D3401A6084D0486063E078DA
:1083B000401CE070C948FEF75FFCE083CC480C909D
:1083C000C4484E300B901630019022E201209BE70A
:1083D000C248FEF751FCE083C64EC74F21E0A07AA9
:1083E000002813D001F07FFD039988420ED9069929
:1083F00088420BD201F04EFC2573099801F0ABFDC9
:10840000012001F0FFFD2072A57211E0B348FEF7D4
:1084100033FC80B2E083618C884202D3C919884260
:1084200006D300210F2001F017FD3042E062D6D0C4
:10843000E06A411C1FD040047ED58122D201002178
:108440000F2001F04EFE0021102001F005FD410635
:10845000A048490E002250300A9101F033FD00205F
:1084600001F09AFD002001F04CFD9A485030417A0D
:108470000729AAD101E0FFF713FF964802229F497E
:108480005530FCF79FFE00289FD100273E460DA8DF
:1084900001F02FFD04200DAA390E36020E433902D9
:1084A000175C0F43401EF7D5A764E66400273E46DD
:1084B000104601F010FD04200DA93A0E36021643B5
:1084C0003A020F5C1743401EF7D527656665A17811
:1084D0006A46491CA1707F494D310E79167749795A
:1084E00051770091607B00280AD1012079492071E1
:1084F000928BCE310A8060710298067500994175A1
:1085000074486946CE3000888F8BB8427ED10B9973
:108510007B48098A01806F4826464C30808A208338
:108520006E48FEF7A9FBF083308B7649FF30C330ED
:1085300080B23083884200E060E10CD949424018A3
:108540006F49308308886F4A401C80B20B32088024
:10855000904200D30D806C49032008700B985B4A51
:1085600081891186C089684B5086903B326B1A60B6
:108570001A46B03AD37C1F073F0F032F00D0B774C1
:108580001A09F274F5700127504AB7729186D086A5
:108590007079FF21913148435A49326D5939401859
:1085A0000104C817736D891858410206080A104360
:1085B00056490990401803901921099889024018DA
:1085C000069009983446B843010E0002F165B06583
:1085D0004048F36C0A30B26C01F0E6FD3D48736D23
:1085E0001630326D01F0E0FD3A48F36D1230B26D95
:1085F00001F0DAFD374808214172707900228000CD
:1086000034491C3001F098FD707900E09BE0800057
:1086100000211C3001F0A2FD2E492C48F7720422E3
:1086200051314030FCF7AAFD3548318B07887D2059
:10863000C00078434018B0630D9035480078F0735F
:1086400006462B484038C088FCF7FDFF05903846A9
:10865000FCF7F9FF0599FCF71BFE7F21C905FCF724
:10866000BEFDFDF719F881B22948761E0180B1429E
:1086700001D10120E072A78414202646205EFCF779
:10868000E9FF07910890F08BFCF7F8FF214A224B95
:10869000FCF7EEFE074600910D98FCF7DBFF3A462B
:1086A000009BFCF7D7FE079B089AFCF72FFEFDF70F
:1086B00007F8F0631948008800F0CAFAF07C002837
:1086C0007ED00C99098881427AD029E048000020A8
:1086D000BC0000209411002000040050A4140020CD
:1086E000666666666666E63F00000840A086010092
:1086F000600D002000D02724983A0000D800002008
:10870000E0000020E70300002413002000AEFCFF7F
:10871000D4000020F853E3A59B843E40C400002011
:108720000C98E17C01801222B8480199FCF726FDE3
:108730000822B649B648FCF721FDB449B4480A22DC
:10874000083130305AE13846FDF7E6FA627B2146BF
:1087500090420CD301220A714A794300521C4A719B
:10876000AA4ACE3AD752029A1675009B5375A74A69
:1087700003230C3A13540B9AA64B96891E86860047
:10878000D289A2485A86096B9C388151B038C27C84
:10879000A37C1107090F994202D9032900D0A274C2
:1087A000E17C2746002914D002229B49401DFCF79A
:1087B00009FD00280DD1012098493874C87100E0E6
:1087C00027E00A981638C2B27A7490480199FCF7EB
:1087D000D5FC92487B6D301816303A6D01F0E4FC00
:1087E0007879002280008D491C3001F0A5FC787951
:1087F000002180001C3001F0B1FC0AE0324600216B
:108800000F2001F06EFC207B002802D0002001F038
:1088100078FBE08B618C884200D2D9E5804A8918C8
:108820008842FAD87F48008881004018E178884261
:1088300000D2A5747C4A00210F2001F052FCA078E0
:108840006071724800260C380078002812D1206C24
:10885000FDF722FB0746754801883846FCF748FCBF
:1088600073487F1E0088414388B27249088067833D
:1088700000F0EEF90020A073617B22798A1822E0D3
:10888000624B0C3B195C00291BD0A57BB3006D1C0F
:10889000A5735E4D9C463C3DE9505C4B4500CE3B8C
:1088A00077005D5B1833DD5385001A33574F5D59F0
:1088B00063466C3FFD50761C3B466033491EF6B262
:1088C0001954401CC0B28242DAD8A078032801D2E1
:1088D000A07BA0734F490022887B48730390401E01
:1088E00031E000212BE0494C8B006C3CE6581D190F
:1088F00006956D68AE4220DDB646444E4C00B63E4D
:10890000365B9700B446414E3C3EF65907963F4EC3
:108910006C3EF55035464A3D67197D884A3E3553D1
:1089200034467A341C197A366568F550069B7646CB
:108930005E6066467E80079E6660491CC9B28142C1
:10894000D1DB521CD2B28242CBDB324800214172D1
:10895000039C2BE02D4B2D4ACE3B4F00B63AD25B09
:10896000DA531D468A0062351E46AD583236B55080
:10897000314EB54218D01D469235AD580A2D13D14F
:10898000457A0626AC4675431E461A3EFB18AE19BC
:108990001B88B3801D4B65469C3BD2181388F3801F
:1089A000528832816D1C4572491CC9B2A142D1D393
:1089B000164B0021204C9C3B8A00491CC9B29C509C
:1089C0000C29F9D3007C002805D0104908784B7891
:1089D0008A7802280ED0144A002180320F2001F03C
:1089E00080FB01210520002249020007FDF79BFFC3
:1089F0000FB0F0BD0648C91C801FC018FCF7BEFBB5
:108A000001F01CFD642000F0C3FF34E530130020AA
:108A1000260D002048000020D800002094110020DE
:108A2000983A0000CC00002000D02724C800002085
:108A3000C6000020C4000020FFFF010070470000B6
:108A4000F8B535493348086001F098FCFF20334DF4
:108A500016306880E888002801D16420E88030481A
:108A60000178432901D943210170E98E01702D4C11
:108A7000E88F2071A88F6071A87AA070A8880090F4
:108A8000E0612889FCF7FAFD274A284BFCF7F0FC47
:108A900000F01AFF0022264BFCF738FCFCF734FEEE
:108AA00086B26681EF8831463846FCF721FBA0810B
:108AB00001460098FCF71CFB71438EB27D20C0007C
:108AC00026817043FCF7DAFD1A4A1B4BFCF738FD90
:108AD000FCF71AFEE0817D2066823946C000FCF773
:108AE00007FB2082E08201202083FDF729F9A08284
:108AF000E28912491248FEF7C3F812A0E16900F0BA
:108B000031FDE98813A000F02DFD298916A000F0A1
:108B100029FDF8BD5994000844000020200D0020D4
:108B200000000020BC000020666666666666E63FC0
:108B300000000840F853E3A59B843E40FF7F0000FF
:108B4000A4140020B1EAC7A949443A202564202E84
:108B50000D0A0000CDA8D1B6BCE4B8F43A202564D3
:108B6000206D732E0D0A0000B5A5B4CECDA8D1B6E8
:108B7000BBF9D5BECAFDC1BF3A202564B8F62E0D9B
:108B80000A00000070B586B014216846FCF70FFBA0
:108B900001250F4EED03002229463046FDF7C3FEA6
:108BA0000120002401900294694600950394304608
:108BB000FDF7F8FD032001900294694600950394A7
:108BC0003046FDF7EFFD022000F0E2FE06B070BD7A
:108BD0000004005070470000F8B5044600206A46C3
:108BE0001080194D55222A70AA226A700322AA7099
:108BF000661DEE702A716971144A49008918AC71BA
:108C00002246E81DFCF7BAFA002007E029186A4658
:108C10008978128889186A461180401CB042F5DBB9
:108C2000611DA81CFCF706FF014668460180291952
:108C30000078C871684640780872214609310248B8
:108C400000F06AFAF8BD0000E4130020200D0020B7
:108C500010B513490A8BCB8A9A4201D3D21A0A83E0
:108C6000104A098BD2884A437D211018C900484315
:108C70000D490968401AFCF7EDFC0C4A0C4BFCF757
:108C80005FFCFCF71DFD0B49884201DD4A4280185C
:108C9000002800DA401808490968486110BD000042
:108CA000BC000020200D002084000020F853E3A524
:108CB0009B843E40FF7F0000A4140020034A1168FB
:108CC000382389B299430143116070470030014055
:108CD00010B5FDF735FE10BD10B59AB034216846C9
:108CE000FCF765FA14210DA8FCF761FA1C2112A803
:108CF000FCF75DFA1B4801680324E402A143C21497
:108D000089180160FEF710F817480169A143016155
:108D100006200090FF2001300290012003901020D7
:108D200004900220099040040B90000100240C9054
:108D30000A946846FEF7F6F90F200D9003200E9076
:108D40000F941094012111940DA8FEF7D9F88120F9
:108D50001290032080041890149412A8FEF71EF8B5
:108D60001AB010BD00700040401002401048016869
:108D7000821511430160C1680E4A1140C16001684B
:108D80000D4A11400160816849084900816001680D
:108D90000122920491430160C168FD2212049143B3
:108DA000C1600021016106490448886070470000E5
:108DB000001002400C40FF88F6FFF6FE005000084D
:108DC00000ED00E070B501F05BF80D4C0D4D6064F6
:108DD00002E001F055F86064A842FAD10020E08278
:108DE0002078002809D0012802D0022805D102E00D
:108DF000FCF7C2FF01E0FFF761FA00F033FF70BD3E
:108E0000480000203001CADE10B5818CC90707D0A8
:108E100001684A6801235B049A43836A1A434A60E3
:108E2000818C890707D501684A6801231B049A438E
:108E3000C36A1A434A60818C490707D501684A68AA
:108E400001239B049A43036B1A434A60818C0907F0
:108E500007D501684A680123DB039A43436B1A4331
:108E60004A60818CC90607D50268916801231B03FB
:108E70009943836B19439160818C890607D50168FA
:108E80008A6801235B039A43C36B1A438A60818C0F
:108E9000490612D503685A6801210905046C8A4302
:108EA00022435A60026C8A4207D102685168032348
:108EB0005B059943436C19435160818C090607D5C2
:108EC00001684A680123DB04806C9A4302434A60CC
:108ED00010BD0000F8B500260446C667FDF72AFD60
:108EE000054620680068124F000709D501212B466E
:108EF000002249052046009700F054FA00280DD1C1
:108F00002068006840070BD501212B460022890507
:108F10002046009700F046FA002801D00320F8BD53
:108F200020206067A067603426740020F8BD000030
:108F3000FFFFFF01F8B5184CC826E078002829D1BA
:108F40006079002826D101206071144D686B0027DC
:108F500000281ED0686BC821081A15E01048E16887
:108F6000405C616988470F480A21008848430E49E0
:108F70000880E068401CE060E068C82800DBE7602B
:108F8000696BC820401A761EE168814201D0002E2C
:108F9000E4DC6771F8BD00003000002000000240F2
:108FA000580C0020CC000020D600002070B5224CC8
:108FB000E07800283FD1207900283CD101202071A1
:108FC0001E4EF16900250906002933DA2156625741
:108FD00091420AD1F06940062CD5A079002829D009
:108FE000A5712089401C208124E0A179002903D1AA
:108FF000A0710A2000F0D3FC00202056CC21484369
:109000000F494218206912181279B262401C0022DE
:109010002061A256CC235A43895881420ADC25613B
:109020002078401C207020780E2800D12570A07870
:10903000401CA070257170BD300000200038014038
:109040003001002010B5806A0022014640314A8379
:109050004A82FEF7FAFA10BD70B5846A606FA56F98
:109060002168896800260906002906DA212804D12A
:1090700052200653204600F047F8206880684006DA
:1090800006D5222D04D15A200653204600F02CF894
:10909000E06F10210843E0672046FEF7D6FA70BD66
:1090A00010B501460968806A0968890614D400224F
:1090B0005A210A5201680A68FF2301339A430A6061
:1090C00001688A68520852008A6001688A684023F1
:1090D0009A438A6020218167FEF752FC10BD10B5CB
:1090E000806AFEF74EFC10BD01680A68FF23213339
:1090F0009A430A6001688A68520852008A602021F7
:10910000816700210166704701680A68C0239A439D
:109110000A6020214167704770B5164CE278002A3A
:109120000CD12279002A09D10122E2700025C82938
:1091300003DC0222A256002A01DCE57070BD012387
:10914000E356CC2253430C4AD1500123E356CC269C
:1091500073439B180A460146181DFCF70FF8607808
:10916000401C607060780E2800D16570A078401EA9
:10917000A070E2E73000002030010020F8B504467E
:109180002669A268E76932436669102000253E43DC
:109190002368324378491E68784F3E4016431E606C
:1091A00023685A6803263603B243E66832435A609E
:1091B0002368A2698B4201D0266A32439E680B273E
:1091C0003F02BE4316439E606D4E23686D4AB34214
:1091D0000CD1D2689207920F06D0012A38D0022A09
:1091E00034D0032A20D11EE001201DE0664EB34298
:1091F0000AD1D2680C26324026D0042A28D0082A68
:1092000024D00C2A10D10EE08B420DD1D668032257
:109210009202164018D001229202B61A18D0B61A3D
:1092200014D0964200D10820564A0126403A574FA2
:10923000F6038B4236D100280CD002280DD004282A
:1092400012D008281FD11CE00020EDE70220EBE738
:109250000420E9E7FDF70AFF08E01068C00601D521
:10926000384605E04A4803E0FDF720FF002873D0A8
:10927000626851005118814205D81103814202D31E
:1092800003E03046F4E7012566E0010E06025008CF
:10929000002330185941FBF741FF03210902411A0D
:1092A0003C4A55E0E169B14232D1030000F081F956
:1092B00009070A0D06250606062B0600E3E7FDF75B
:1092C000D5FE1CE0FDF7E2FE19E010686168C006FB
:1092D00002D54808304A01E0304A48088018FBF7B8
:1092E00007FF80B201462E4A10399142CBD8511C5B
:1092F00001400007400F08432CE0FDF7D7FE6168EE
:1093000040004A08EAE76168012248081204E5E7DC
:10931000030000F04EF909070A0D06260606062C82
:109320000600B0E7FDF7A2FE1DE0FDF7AFFE1AE074
:1093300010686168C00602D54808C01902E01448E8
:109340004A081018FBF7D4FE80B20146144A1039BF
:10935000914298D82168C86000202066606628463F
:10936000F8BDFDF7A3FE61684A088018EAE7616866
:1093700048088019E6E7000000480040F369FFEF65
:1093800000380140401002400044004000093D0008
:109390000024F400FFFC0F0000127A000048E801EE
:1093A000EFFF0000FFB581B017460E4604460A9D48
:1093B00009E0681C07D0FDF7BDFA0499401AA842DD
:1093C0000CD8002D0AD02068C1693046884318D0D7
:1093D0000020B842EDD0002005B0F0BD2068016843
:1093E000FF22A13291430160206881684908490049
:1093F000816020206067A067002060342074032013
:10940000EAE70120E5E7000010B5044910200968EB
:1094100008620248FEF71AF910BD00002C15002062
:1094200001490D20887070473000002010B50748B2
:109430000A22018A51434183FEF7F4FDFEF7D6FE6E
:10944000C82203490348FEF73FFA10BDBC000020C4
:10945000580C00202C150020F8B53D4C0023217835
:109460003C4A1D46082910D0072945D006294ED070
:10947000052950D0042951D0032952D0002954D0B5
:10948000012956D0022958D059E0A17800264A1F58
:1094900004E0304FBF5DFB189BB2761C9642F8DBB0
:1094A000667927799A195118E3786278C91889186A
:1094B000C9194018C0071AD0012E14D0022E16D197
:1094C00025482449C018FBF759FE00F0B7FF642077
:1094D00000F05EFABFF34F8F21492048C860BFF308
:1094E0004F8F00BFFDE759081046FFF775FB257049
:1094F000E570A570A571F8BDA1795054491CC8B29A
:10950000A071A178491F8842F5D1082001E0607060
:1095100007202070F8BDE0700620FAE76071052092
:10952000F7E7A070E5700420F3E7552807D1012084
:10953000EFE7AA2803D10220EBE7032803D0257028
:10954000E570A570F8BD032020702071F8BD000003
:10955000B300002080130020200D00200400FA0535
:1095600000ED00E00FB410B503A9044B044A0298C3
:1095700000F002F910BC08BC04B01847C1A10008F3
:10958000F00000202021020C01D010211046020A18
:1095900001D010460839020901D01046091F82087F
:1095A00001D01046891E420801D0881E7047081A53
:1095B000704730B47446641E2578641CAB4200D2F8
:1095C0001D46635D5B00E31830BC184702E008C825
:1095D000121F08C1002AFAD170477047002001E02D
:1095E00001C1121F002AFBD1704708B5002168464F
:1095F00001706B46012202212C2000F081FD022126
:10960000684601706B4601222C2000F079FD08BDF0
:1096100038B504466D20694608706B46012207493B
:109620002E2000F06DFD0649002C01D0054A00E017
:10963000054A2E2000F04AFD38BD00000608000053
:1096400006180000070600000716000038B504469B
:109650006B4602220021362000F018FCB3212300C3
:10966000FFF7A7FF0E0F08153A3A3A3A1C273A3A85
:109670002F34483A0021684601704078410849007B
:1096800014E06946087880088000401C04E06946C0
:10969000087880088000801C08701DE06846027809
:1096A0000A40483202704178802001436846417088
:1096B00012E0684602780A40027040784106490E7E
:1096C000F4E7694648780221084303E06946487890
:1096D000FD210840694648706B4601220021362072
:1096E00000F00EFD012200AB11463620013300F0E0
:1096F00007FD38BD69460878CF210840694620300B
:10970000CAE708B5032168464170012101706B4624
:1097100002220021362000F0F3FC0122D2030621B0
:109720002D2000F0D3FC012000F032F90120FFF7DA
:109730008DFF08BD08B5020A69464A7008706B467D
:10974000022204212D2000F0DBFC03206946087072
:109750006B46012206212D2000F0D2FC0020694634
:1097600008706B46012206212D2000F0C9FC0A2159
:109770002D2000F071FB08BDFFB58DB0044600251B
:1097800006E025280AD0109A0F999047641C6D1C9A
:1097900020780028F5D1284611B0F0BD002701211E
:1097A000484A009700E00743641C23780846203BA2
:1097B00098401042F7D120782E2817D10420074373
:1097C0006078641C2A280CD10E98641C02C8009191
:1097D0000E900BE000990A22514330394018641C66
:1097E00000902078014630390929F3D920780028E3
:1097F000D1D0642808D0692806D075281ED0109AC8
:109800000F9990476D1C5BE00A200E99019001C9E9
:109810000E91002802DA40422D2102E0390504D5DC
:109820002B216A461172012103E0F90704D020219F
:10983000F7E70BAE0B910DE00021FAE70A200E9935
:10984000019001C90E91F7E70199FBF751FC303106
:10985000761E31700028F7D103A8801B20300190BC
:10986000780701D5009801E0012000900199884215
:1098700001DD401A00E000200027009006E002A869
:10988000109AC05D0F9990476D1C7F1C0B98874202
:10989000F5DB04E0109A30200F9990476D1C009979
:1098A000481E00900029F5DC05E03078109A761CFF
:1098B0000F9990476D1C0199481E01900029F4DC16
:1098C000641C65E709280100F8B54A002B4B520DCE
:1098D000D6182B4A0C460546142E2BDA002E12DA27
:1098E000284BFBF713FD00221346FCF739F840D252
:1098F000002C03DA0124E40700253AE0204628433F
:1099000037D0214C14E0214F0B46F7403B402B430E
:1099100031D01C4BFBF7FAFC00221346FCF720F871
:1099200027D2002C03DD01200005F0400419BC43C0
:1099300000251EE0332E1EDC33460027143BFF4378
:10994000DF40384217D00F4BFBF78AFD0022134649
:10995000FCF706F80DD2002C0ADD142E0CD03420B2
:10996000811B012088404019A84200D2641C054692
:10997000BD4321462846F8BD641CF9E701FCFFFF02
:109980009C7500883CE4377E0000F03FFFFF0F002D
:109990007D2110B5C900484300F001F810BD002139
:1099A00040E000BF00BF00BF00BF00BF00BF00BF5E
:1099B00000BF00BF00BF00BF00BF00BF00BF00BFAF
:1099C00000BF00BF00BF00BF00BF00BF00BF00BF9F
:1099D00000BF00BF00BF00BF00BF00BF00BF00BF8F
:1099E00000BF00BF00BF00BF00BF00BF00BF00BF7F
:1099F00000BF00BF00BF00BF00BF00BF00BF00BF6F
:109A000000BF00BF00BF00BF00BF00BF00BF00BF5E
:109A100000BF00BF00BF00BF00BF00BF00BF00BF4E
:109A200000BF491C8142BCD370470000FEB504460C
:109A30000020019000906079734940000E5A6178CF
:109A40002578491E7148CFB20163042D77D0072DC8
:109A500075D000210291217801736C49E3790122CC
:109A600092058969002B6CD0914381616748217A06
:109A70004173217A82698907890B0A438261002137
:109A8000042000F02EFB324661492E2000F01EFB20
:109A90003846FFF7BDFD5F4E0522705D810040181E
:109AA0005D49431807212B2000F02AFB5B490298EF
:109AB00001220B180B21282000F022FB705D584971
:109AC00080000A580C21282000F00BFBE079554952
:109AD00080004018A1794900425A0221272000F055
:109AE000F5FA51487E00825B0421272000F0EEFA4F
:109AF000E079002829D0A07804282CD028206946B5
:109B0000087220220621272000F0E0FA02AB012291
:109B10002621272000F0F4FA444938014018E17862
:109B2000890042580821272000F0DBFAA17A601C46
:109B3000627A0902114313D016E000E001E001212E
:109B400088E71143F608816190E764220621272007
:109B500000F0BCFAE0E71020694608720246D1E73F
:109B600033490172090A4172417A007A0A020243BA
:109B70002021272000F0AAFA2E4F0C2123203A683A
:109B800000F0AFFAF01982880421232000F09EFA39
:109B9000A07900280BD0E079274901224318002141
:109BA000212000F0ADFA03200190012000902A0747
:109BB000120F10010243607800218007000B02435E
:109BC0000198000502430098400402432079C00632
:109BD000400902436079C00602431F2000F081FA69
:109BE000A07861780123084302040848DB0302617E
:109BF000E179490319430A4302610021082000F07A
:109C000070FA0020FEBD000008A50008F400002046
:109C100004280000B0A40008010000201F0000205C
:109C2000B8A40008D8A40008E4A40008E8A4000828
:109C300041100000D0A400082100002038B50C46D7
:109C400007498A8B002102432C2000F03FFA684626
:109C500004706B46012206212C2000F051FA38BD19
:109C6000F400002010B5FFF7C0FC10BD10B504468D
:109C70000421362000F0F0F80121C902002C01D0A7
:109C8000084300E0884302460421362000F029FA08
:109C900010BD000038B540206946087000210E2034
:109CA00000F0DAF80446002211460E2000F019FAFE
:109CB0006B46012200210D2000F022FA074A002104
:109CC0000F2000F00EFA00F0E7F9224600210E20E6
:109CD00000F007FA02480021017338BDF8FF27247D
:109CE000140100207CB505460420694608704B4CE1
:109CF0000020607521462031206348710873A083DD
:109D00006063A06300F0BCF8454E206002E000F004
:109D1000B7F82060B042FAD10020FFF797FC414825
:109D20000078242801D9243806E00621FBF7E0F961
:109D30000622101A40010843020601040A430102E8
:109D40000A43024300211E2000F0CBF96B4601229A
:109D50000021242000F0D4F91E20FFF7EBFC86B28E
:109D6000300AA0730420FFF7E5FC0006000E0DD0BA
:109D700002206946087101AB012212212D2000F05A
:109D8000BFF9A08B012109030843A08300F078F8F4
:109D900020600620FFF7CEFC60600720FFF7CAFCBA
:109DA000A060F006C00E207501D110202075C0B251
:109DB00000F0E2F9E80707D0FFF7A3FCA08B012130
:109DC000C9020843A0830AE00521362000F02EF8DE
:109DD0001549084002460521362000F077F9012098
:109DE000FFF734FC0021042000F036F8A0610021C8
:109DF000262000F031F8152189030843024600218E
:109E0000262000F06EF900222621362000F05EF9AF
:109E100000F036F8206000207CBD0000F400002037
:109E20003001CADE00000020FFFD000038B5094CFB
:109E300089B280B26B46022200F028F8002806D1D1
:109E400068464078010268460078081884B22046C7
:109E500038BD0000FFFF000038B50024E44389B29C
:109E600080B26B46042200F011F8002806D10321CD
:109E70006846435C2202D418491EFAD5204638BDF4
:109E800010B500210846FFF7E7FF10BD38B50029DF
:109E900009D0402420436C462070C8B27F2906D8E0
:109EA000607002200AE069460870012006E0802404
:109EB00020436C466070C809A0700320694600F01A
:109EC00097FA38BD10B5144603460A4621461120BC
:109ED000FFF7DCFF10BD10B5034605220021152059
:109EE000FFF7D4FF10BD10B501210620FFF7B4FF26
:109EF00010BD10B50346052200211720FFF7C6FF4D
:109F000010BD38B5054600206946087000F0C4F859
:109F1000FF2401342246002D01D003221202002129
:109F20000D2000F0D3F8002D13D06B460122032141
:109F30000F20FFF7ABFF68460078000709D5FFF751
:109F4000A9FE224600210D2000F0C0F80020C043E9
:109F500038BD002038BD10B5024601210A2000F0AE
:109F6000C0F810BD10B5044600211A20FFF774FF99
:109F7000000D22030005120B024300211A2000F0FD
:109F8000B0F810BD10B5024602492E2000F09EF830
:109F900010BD000004180000F8B505466B4601220C
:109FA00003210420FFF772FF0126114C3607002D14
:109FB0000DD02A4600210C2000F088F86946087868
:109FC0001021084369460870A069304307E06946DC
:109FD0000878EF21084069460870A069B0430B4635
:109FE000A06101220321042000F08AF8F8BD0000DE
:109FF000F400002010B502460021182000F066F899
:10A0000010BD0000F8B50746002568460570B80782
:10A01000204C2E4600280ADA8020694608706B46DC
:10A02000012200210D2000F06BF801202073F807B9
:10A030006946087821D006210843694608706B46B6
:10A04000012200210D2000F05BF803210F20FFF713
:10A05000EDFE8121C900084219D0402069460870F0
:10A060006B46012200210D2000F04AF80020FFF786
:10A07000FDFD00252673ED4309E0022108436946F2
:10A0800008706B46012200210D2000F039F82846A7
:10A09000F8BD0000140100201CB56B46012203210D
:10A0A0000F20FFF7F3FE684600784022C1091040F8
:10A0B000C9014000814208D001206946087102466A
:10A0C00001AB03210D2000F01BF81CBD08B56B4649
:10A0D0001A70120A5A7089B280B2022200F010F887
:10A0E00008BD38B500236C46E254120A5B1C042BF1
:10A0F000FADB89B280B22346042200F001F838BDB1
:10A1000038B58024002909D0C02528436D46287021
:10A11000C8B27F2907D86870022009E02043694649
:10A120000870012004E020436870C809A87003206B
:10A13000694600F099F938BD10B51446012312188C
:10A140009B029A4202D90020C04310BD0B46821EDA
:10A1500021460920FFF7D4FF002010BD10B5054AA5
:10A160008905126901430A4300210820FFF7B9FF5E
:10A17000002010BDF400002038B504466B460122D3
:10A180000E212B20FFF782FE68460078E106400989
:10A190004001C90E0143684601706B4601220E2141
:10A1A0002B20FFF7ADFF38BD10B5002142541C062F
:10A1B000120A22431B0A491C0429F7DB10BD0000C8
:10A1C00013B501231A4669460248FDF7DBFB0098E8
:10A1D0001CBD00002C150020FCF7BAFBFEF77CFD2F
:10A1E000FDF734FF3F494048002522C005608561E6
:10A1F000C5613E490562C1600838FCF7C3FCFDF744
:10A2000011FFFDF7F3FFFDF7CFFFFDF7D7FE0526A2
:10A2100001223607D1033046FCF785FBFEF710FC20
:10A22000FDF7D0FDFBF75CFCFBF734FC0721B01514
:10A23000FFF704FDFFF716FD2D4C0A21208A0122AD
:10A240004843608311033046FCF76DFB2648C82263
:10A2500028498830FDF738FB274F284EE078002842
:10A260003CD0FEF739FDE570FBF74EFE20700F285D
:10A270000AD9012211033046FCF755FBFEF7A2FD77
:10A2800000220121090309E0012251033046FCF7B5
:10A290004AFBFEF797FD0022012149033046FCF7F7
:10A2A00042FBFDF7D9FC608B002801D0401E608383
:10A2B0001348618B00780843D0D13878002801D04A
:10A2C0000328CBD10121C9023046FCF727FB002827
:10A2D000C4D101210846FCF747FDBFE7FDF7BCFCF0
:10A2E000BCE70000007C0040A4140020FFFF000039
:10A2F000BC000020580C00205A0000200004005030
:10A300003600002010B586B01748FCF7C0FB1421BA
:10A310006846FAF74CFF1548009003200190002092
:10A320000290052069460007FCF73CFA6946104890
:10A33000FCF738FA69460F48FCF734FA0121084661
:10A34000FCF712FDFF2401342046FCF7E5FC0A4926
:10A3500008680422104308602046FCF7EDFCFCF777
:10A36000F3FC06B010BD0000A4140020FFFF0000A5
:10A3700000040050000800500070004010B5012299
:10A38000920218491848FBF721FC16481749028821
:10A390008A4225D0018004218180FF21F531C180CE
:10A3A0000A21018100211E224181D24382810122A2
:10A3B000C2810184018241828182C18201838183C1
:10A3C0004323C38602230387782343878287C28778
:10A3D00002464032118451849184C18300F02EF8EA
:10A3E00010BD0000200D002000FC0008AA55000050
:10A3F000F0B58C4600251026052109078E620E4C0B
:10A4000008E067467F5DE760A768FF07FCD0E76864
:10A410001F706D1C8542F4DB0020074606E0E760F4
:10A42000A568ED07FCD0E5681D54401C9042F6D3AA
:10A430008E610020F0BD00000030014070B572B6A2
:10A440000124074DA40221462846FBF7A5FB00285E
:10A4500004D0224603492846FBF742FC62B670BD91
:10A4600000FC0008200D0020F0B50025102605276F
:10A470009C463F070B46BE620C4C06E0595DE1600E
:10A48000A168C907FCD0E1686D1C8542F6DB00209D
:10A4900007E06146095CE160A168C907FCD0E1689A
:10A4A000401C9042F5D3BE610020F0BD0030014059
:10A4B0000000010203040005405C0000A05C0400F1
:10A4C000C06C0800805C0400E03F1E00E07D1E00C0
:10A4D00007A9022570889B880A0016000100060063
:10A4E0000100020087008D002D001A3152001A333E
:10A4F0009A001A351D011A376B003B31BE003B3301
:10A500005E013B3596023B37000099599959EB5152
:10A510008F421E45142E0080EB51F5283333E13A6B
:10A52000703DE13AC235852BC2353333C235C23571
:10A53000AE47E13A5138A330513800000000000026
:10A5400000000102030406070809030406080C10B2
:10A550001820300000000001020304007CA5000860
:10A5600000000020F4000000CC95000870A6000850
:10A57000F400002064190000DC95000800070400C6
:10A58000091E08054008260910400856080540081D
:10A59000261D040008BE1D040008BED8BC401008DB
:10A5A000010000000000C8420000000000000000A0
:10A5B000000000000000000000000000000000009B
:10A5C000000000000100000000000000000000008A
:10A5D00000000000000000008C0A000000000000E5
:10A5E000000000000000000000000000000000006B
:10A5F000000000000000000000000000000000005B
:10A60000000000000000000000000000000000004A
:10A61000000000000000000000000000000000003A
:10A62000000000000202140009090102008100007C
:10A630000000000001000000000000000000000019
:10A64000000000000000000000000000000000000A
:10A6500000000000000000000000000000000000FA
:10A6600000000000000000000000200000000000CA
:04000005080050C1DE
:00000001FF
